:10000000A220A200A203A20078A960853F203F00A1
:10001000BABD0001588DF807290F853FA80A0A0AC2
:100020000A853EAA2CFFCFA000B916C9F00D0980A1
:10003000995007C810F3A9C520A8FC2C61C0100B6B
:10004000ADF8073A854164406C40002000C8C90003
:10005000D0EEA9088545644464476446207CCAB054
:10006000DFA90A854564446447A9018546207CCA06
:10007000B0CE4C01081890013808FAA004B93D0030
:10008000488810F9863D78A960853F203F00BABDB9
:100090000001588DF807290F853FA80A0A0A0A852A
:1000A0003EAA2CFFCF203DCA9004A92F8015A9801D
:1000B0003C83C0D0052000C8B009A53D4828B03415
:1000C0002055CADAA63F9D7804689DF804989D786B
:1000D0000508689DF805A00068993D00C8C0059016
:1000E000F7BDF80548BD780548BDF80448BD78045B
:1000F000FA7A2860182056CB80C900000000977556
:10010000A9039D81C0BD83C009019D83C0A9079D2E
:1001100082C0A00AA9FF9D80C03C81C010FB88D08E
:10012000F5BD83C029FE9D83C0A93D8540A9C98531
:1001300041206DC92081C9C901D065A9498540A95F
:10014000C98541206DC92098C9C901D056A43FB9BD
:10015000F805C9AAD04AA9558540A9C98541206D8D
:10016000C92081C9A9618540A9C98541206DC920DF
:1001700081C9C901F0E0C900D026A95B8540A9C9A1
:100180008541206DC92098C9C900D014A43FB97811
:10019000042940F048BD83C009109D83C04CEFC8BE
:1001A0004C04C9A9558540A9C98541206DC9A967D5
:1001B0008540A9C98541206DC92081C9C901F0E3E5
:1001C000C900D0034CDDC8A9438540A9C985412099
:1001D0006DC92081C9C901F0F6C900D027A94F8592
:1001E00040A9C98541206DC92081C9C900D015BD6C
:1001F00083C009809D83C0BD81C009049D81C01852
:10020000A000900338A027BD83C009019D83C0A929
:10021000009D82C0986020204170706C655D5B53CA
:10022000642076312E32202863293230313820463E
:100230006C6F7269616E20526569747A00400000CB
:100240000000954100000000F948000001AA875015
:1002500000000200FF7700000000FF7A00000000AD
:10026000FF6940000000776900000000FF5AA0000D
:10027000B1409D80C03C81C010FBC8C00690F17A9F
:1002800060A9FF9D80C03C81C010FBBD80C030F1E3
:1002900048A9FF9D80C068602081C9485AA0044CCD
:1002A000A7C9A9FF9D80C03C81C010FBBD80C0488C
:1002B00088D0EFA43F6899F805689978056899F89F
:1002C00004689978047AA9FF9D80C06860DA5AA60C
:1002D0003FA43EA5469DF805A5479D78059EF804D8
:1002E0009E78049845432970F005A9029DF80424DE
:1002F000431007BDF8041A9DF804A9103983C0D033
:1003000011A0091EF8053E78053EF8043E780488E1
:10031000D0F17AFA605AA43F9D80C0B978049D80DC
:10032000C0B9F8049D80C0B978059D80C0B9F805B2
:100330009D80C0A9FF9D80C02081C97A6048A940E6
:100340003C83C018F00138686048A9203C83C0187D
:10035000F001386860A542F00CC901F00BC902F049
:100360000AA90138604C6ECA4C7CCA4CE5CAA90087
:100370002049CA9002A92BA2FFA0FF6020CDC9BDD1
:1003800083C029FE9D83C0A9512015CAC900D05041
:10039000A9FF9D80C0BD80C0C9FED0F4BD81C00949
:1003A000109D81C0A9FF9D80C0A000BD80C0914468
:1003B000C8D0F8E645BD80C09144C8D0F8C645BD58
:1003C00080C0BD80C0BD80C0BD81C029EF9D81C0FF
:1003D00018A9000848BD83C009019D83C068286032
:1003E00038A92780EE2049CAB06720CDC9BD83C097
:1003F00029FE9D83C0A9582015CAC900D04EA9FF67
:100400009D80C0A9FE9D80C0A000B1449D80C0C851
:10041000D0F8E645B1449D80C0C8D0F8C645A9FFD4
:100420009D80C09D80C09D80C0BD80C0291FC90522
:10043000D01A18A5000848A9FF9D80C0BD80C0F053
:10044000F6BD83C009019D83C068286038A9278054
:10045000E438A92B80DFA004B94800488810F9BA15
:10046000BD0D0185481869039D0D01BD0E0185492B
:1004700069009D0E01A001B1488542C8B148AAC8D3
:10048000B14885498648A901A642E00AB01AB24897
:10049000DDECCCD027A001B148A43F9978068A0AA8
:1004A000AA20C0CBB002A900AAA00068994800C841
:1004B000C00590F78AA002A200C90160A90480E8E3
:1004C0007CF6CC2051CCA43FB97806D018A54CF0CE
:1004D00004A9213860A904924AA007B909CD914A1C
:1004E00088D0F81860A64CF016CAF008CACAF00FF7
:1004F000A9213860A901924AA8A900914A1860A9C7
:10050000E8A63E203DCAB00209102049CA9002095F
:1005100004924AA001A9FF914AC8914AC8A9009132
:100520004AA54CF00CA004B90DCD914AC8C0199051
:10053000F618602051CCA64CF00FCAF00CCAF00699
:10054000CAF00ACAF003A92138A9001860A91F3807
:1005500060A002B148854AC8B148854BC8B14885FA
:100560004C60207CCC900160A63EA43F4C7CCA200D
:100570007CCC900160A63EA43F4CE5CAB97806F059
:1005800044C901F00EC902F00EC903F010C904F00D
:10059000118032A53E8010A53E0980800AA53E3A12
:1005A0008005A53E3A09808543A002B1488544C82C
:1005B000B1488545C8B1488546C8B1488547C8B1E6
:1005C00048D0061860A9113860A92D3860B978069E
:1005D000F004A9001860A9113860B9780618F00372
:1005E000A9113860A9013860A92738600303030105
:1005F000030101010404C3CB62CC6FCCCDCC33CC5E
:10060000DACCE4CCE4CCE8CCE8CC4000000B12001F
:1006100000104150504C455D5B5344202020202069
:10062000202002000B12000000000000000000006B
:1006300000000000000000000000000000000000BA
:1006400000000000000000000000000000000000AA
:10065000000000000000000000000000000000009A
:10066000000000000000000000000000000000008A
:10067000000000000000000000000000000000007A
:10068000000000000000000000000000000000006A
:10069000000000000000000000000000000000005A
:1006A000000000000000000000000000000000004A
:1006B000000000000000000000000000000000003A
:1006C000000000000000000000000000000000002A
:1006D000000000000000000000000000000000001A
:1006E000000000000000000000000000000000000A
:1006F00000000000000000000000000000000000FA
:1007000000000000000000000000000000000000E9
:1007100000000000000000000000000000000000D9
:1007200000000000000000000000000000000000C9
:1007300000000000000000000000000000000000B9
:1007400000000000000000000000000000000000A9
:100750000000000000000000000000000000000099
:100760000000000000000000000000000000000089
:100770000000000000000000000000000000000079
:100780000000000000000000000000000000000069
:100790000000000000000000000000000000000059
:1007A0000000000000000000000000000000000049
:1007B0000000000000000000000000000000000039
:1007C0000000000000000000000000000000000029
:1007D0000000000000000000000000000000000019
:1007E0000000000000000000000000000000000009
:1007F00000000000000000000000000000000000F9
:00000001FF
